:100000000C9472000C9486000C9486000C9486006C
:100010000C9486000C9486000C9486000C94860048
:100020000C9486000C9486000C9486000C94860038
:100030000C9486000C9486000C9486000C94860028
:100040000C9486000C9486000C9486000C94860018
:100050000C9486000C9486000C9486000C94880006
:100060000C9486000C9486000C9486000C948600F8
:100070000C9486000C9486000C9486000C948600E8
:100080000C9486000C9486000C9486000C948600D8
:100090000C9486000C9486000C9486000C948600C8
:1000A0000C9486000C9486000C9486000C948600B8
:1000B0000C9486000C9486000C9486000C948600A8
:1000C0000C9486000C9486000C9486000C94860098
:1000D0000C9486000C9486000C9486000C94860088
:1000E0000C94860011241FBECFEFD1E2DEBFCDBF3E
:1000F00000E00CBF22E0A0E0B2E001C01D92A930F8
:10010000B207E1F70E94D2000C9470010C94000039
:100110001F920F920FB60F9211242F933F938F933C
:100120009F93AF93BF938091050290910602A09197
:100130000702B09108023091040226E0230F2D3708
:1001400058F50296A11DB11D20930402809305026B
:1001500090930602A0930702B093080280910002D8
:1001600090910102A0910202B09103020196A11D9B
:10017000B11D8093000290930102A0930202B093FC
:100180000302BF91AF919F918F913F912F910F905B
:100190000FBE0F901F90189529E8230F0396A11DFD
:1001A000B11DD2CF789484B5826084BD84B581605E
:1001B00084BD85B5826085BD85B5816085BD809132
:1001C0006E00816080936E001092810080918100AA
:1001D00082608093810080918100816080938100A2
:1001E000809180008160809380008091B100846064
:1001F0008093B1008091B00081608093B0008091C5
:100200009100826080939100809191008160809341
:100210009100809190008160809390008091A10076
:1002200082608093A1008091A10081608093A100F1
:100230008091A00081608093A00080912101826064
:10024000809321018091210181608093210180911F
:10025000200181608093200180917A0084608093E6
:100260007A0080917A00826080937A0080917A008F
:100270008E7F80937A0080917A00806880937A00E4
:100280001092C100D0E0C0E0C036D10579F0C2368E
:10029000D10561F0CE35D10549F060E0CE010E9474
:1002A000620160E0CE0101960E9462012296C115B2
:1002B00080E1D80749F7C0E0D0E02097F1F30E9431
:1002C0000000FBCF262FF999FECF1FBA92BD81BD4A
:1002D00020BD0FB6F894FA9AF99A0FBE01960895C8
:0402E000F894FFCFC0
:00000001FF
